:020000040000FA
:0600000066EF1AF0120089
:0600080004EF08F01200F5
:060018000CEF08F01200DD
:0610000066EF1AF0120079
:06100800A2EF11F012003E
:06101800ABEF11F0120025
:06102A000100EA340000A1
:08103000DC01000013000000C8
:08103800D9CFE6FFE1CFD9FF9B
:10104000E652A098636A626A0F01266B020EE66E92
:10105000E66AE66A270EE66E0F0EE66E3CEC1AF0C4
:101060000B6E050EE15E0B500F01160E396F9F0ED1
:10107000376F7B0E366FDF6ADF500B6E0C6A0C0E1B
:101080000B5C000E0C5810E2DF50040DF3CFE9FFAB
:10109000F4CFEAFF000EE9260D0EEA22EE6AEE6AB0
:1010A000EE6AEE6ADF2AE8D7658C0F01386B659827
:1010B000659C62A607D062960001786B7D6B7E6BA3
:1010C0007F6BF7D70001010E916F926F936B946B5A
:1010D000856BDF6A030EDF5C26E2EA6ADF34FE0B13
:1010E000EA36E96E6E0EE926000EEA22EE6AED6A35
:1010F000EA6ADF34FE0BEA36E96E680EE926000E76
:10110000EA22EE6AED6ADF50EA6A890FE96E000EA4
:10111000EA22EF6ADF50EA6A8C0FE96E000EEA22DB
:10112000EF6ADF2AD7D70001080E6E6F0D0E6F6FC2
:101130000F01160E266F0D01300E026F0D0E036F9C
:10114000080E016F840E006F0001616B606BE55249
:10115000E552E7CFD9FF1200D9CFE6FFE1CFD9FFA3
:10116000E6520001605118E107D0656A0F01366B45
:101170000001606BA198C7D0656A0F01366B160E2F
:10118000396F9F0E376F7B0E366F65B602D065865E
:10119000FCD70001010E606F60050AE165BA08D056
:1011A000626A0F01366B368136890001020E606F6C
:1011B0006250040B07E00F013651040B03E0629408
:1011C000C6EC0EF065A202D0A1989DD06250010B32
:1011D00009E00F013651010B05E02EDF0001040E7E
:1011E000606F62906250100B07E00F013651100BD8
:1011F00003E0B0EC0EF0629862AC1AD00F0136AD8D
:101200000FD0010EE66EE66A000EE66EE66A730E19
:10121000E66EE66AADEC16F00B6E060EE15E0B5064
:10122000629C00018F5101E08F078F5101E1F2D9DB
:101230006250200B06E00F013651200B02E096ECC5
:101240000EF06250020B14E00F013651020B10E059
:10125000010EE66EE66A000EE66EE66AE6687F0E4E
:10126000E66EADEC16F00B6E060EE15E0B50636A97
:10127000040E0001E76E6019E8AE02D0E73402D038
:10128000E750605D02E2A1983ED00F0136A73AD048
:10129000DF6A040EDF5C36E262A631D064CF86F0EE
:1012A00000018651780BE842E842E842876F629677
:1012B00086B508D08751EA6A8C0FE96E000EEA22E3
:1012C000EF7007D08751EA6A890FE96E000EEA22B3
:1012D000EF70875103E1DEEC0EF010D0000EE66EE9
:1012E000E66A860EE66E000EE66E720EE66EE66A40
:1012F000ADEC16F00B6E060EE15E0B5001D002D085
:10130000DF2AC7D7A198E552E552E7CFD9FF1200EF
:10131000D9CFE6FFE1CFD9FF020EE126FD0EDBA417
:1013200007D0E66AFE0EDBCFE6FF05DAE552E552AE
:10133000FD0EDBA208D0010EE66EFE0EDBCFE6FF4F
:10134000FAD9E552E552FE0EDB500C6A260F0B6E01
:101350000F0E0C220BC0DEFF0CC0DDFFDECFE9FF5D
:10136000DDCFEAFFFD0EDBCFEFFF020EE15C02E214
:10137000E16AE552E16EE552E7CFD9FF1200D9CF1D
:10138000E6FFE1CFD9FF020EE126FD0EDB500FE0B4
:10139000FE0EEA6ADB34FE0BEA36E96E6E0EE926D3
:1013A000000EEA22EECFDEFFEDCFDDFF0ED0FE0E07
:1013B000EA6ADB34FE0BEA36E96E680EE926000EB7
:1013C000EA22EECFDEFFEDCFDDFFD9CFE9FFDACFA6
:1013D000EAFFEE50ED1003E1F36AF46A49D0DECF84
:1013E000E9FFDDCFEAFF020EE926000EEA22FB0E3E
:1013F000DBCFEEFFFC0EDBCFEDFFDECFE9FFDDCF75
:10140000EAFFEE52FA0EDBCFEFFF400E0B6EDECF9F
:10141000E9FFDDCFEAFF0B50EF16880E0B6EDECF33
:10142000E9FFDDCFEAFF0B50EF12FD0EDB500CE0C1
:10143000FE0EEA6ADB34FE0BEA36E96E6E0EE92632
:10144000000EEA22EF740BD0FE0EEA6ADB34FE0BCC
:10145000EA36E96E680EE926000EEA22EF74DECF66
:101460000BF0DDCF0CF00BC0F3FF0CC0F4FF00D08D
:10147000020EE15C02E2E16AE552E16EE552E7CF7D
:10148000D9FF1200D9CFE6FFE1CFD9FF020EE12646
:10149000FE0EDB5020E166C0E9FF67C0EAFFEE52B6
:1014A000080EEF6E66C0E9FF67C0EAFF020EE9268C
:1014B000000EEA22300EEE6E0D0EED6E66C0E9FFF4
:1014C00067C0EAFF8C0EEF6E6EC0E9FF6FC0EAFFE7
:1014D000840EEF6E3DD0FD0EDB50E8240D6EFE0E47
:1014E000DB50040DF3500D24040DF3CF0BF0F4CFBB
:1014F0000CF0000E0B260D0E0C220BC0DEFF0CC0F4
:10150000DDFF840E0B6EDECFE9FFDDCFEAFF0B506F
:10151000EF12FD0EDB50E8240D6EFE0EDB50040DC5
:10152000F3500D24010F040DF3CF0BF0F4CF0CF0AA
:10153000000E0B260D0E0C220BC0DEFF0CC0DDFFD3
:10154000840E0B6EDECFE9FFDDCFEAFF0B50EF120A
:10155000020EE15C02E2E16AE552E16EE552E7CF9C
:10156000D9FF1200D9CFE6FFE1CFD9FF65A84ED051
:10157000FE0EEA6ADB34FE0BEA36E96E6E0EE926F1
:10158000000EEA22EE50EFCFEAFFE96E400EEE16B3
:10159000EE6AEE6AEE6AFE0EEA6ADB34FE0BEA36AB
:1015A000E96E6E0EE926000EEA22EE50EFCFEAFF5A
:1015B000E96EEE7CFE0EEA6ADB34FE0BEA36E96E7B
:1015C0006E0EE926000EEA22EF74400E0B6EFE0E40
:1015D000EA6ADB34FE0BEA36E96E6E0EE926000E8F
:1015E000EA22EE50EFCFEAFFE96E0B50EF16FE0E47
:1015F000EA6ADB34FE0BEA36E96E6E0EE926000E6F
:10160000EA22EE50EFCFEAFFE96EEF7CE552E7CF3A
:10161000D9FF1200000191514DE1010E916F9251DD
:1016200049E1010E926F020E755D0DE16EC0E9FF9A
:101630006FC0EAFFEE52EF6A6EC0E9FF6FC0EAFFCB
:10164000C80EEF6E37D0750535E1886B64C0E9FFD1
:1016500065C0EAFFEE52080EEF6E64C0E9FF65C098
:10166000EAFF020EE926000EEA22300EEE6E0D0EA3
:10167000ED6E64C0E9FF65C0EAFF840EEF6E010EF7
:10168000886F66C0E9FF67C0EAFFEE52080EEF6E92
:1016900066C0E9FF67C0EAFF020EE926000EEA22F3
:1016A000300EEE6E0D0EED6E66C0E9FF67C0EAFF0C
:1016B000800EEF6E12000001936B946B020E755D4D
:1016C0001AE166C0E9FF67C0EAFFEE52080EEF6E4E
:1016D00066C0E9FF67C0EAFF020EE926000EEA22B3
:1016E000380EEE6E0D0EED6E66C0E9FF67C0EAFFC4
:1016F000C80EEF6E1FD079510D01365D00017A5191
:101700000D01375904E236CD79F037CD7AF0D1D8D2
:101710006EC0E9FF6FC0EAFF020EE926000EEA2262
:10172000380EEE6E0D0EED6E6EC0E9FF6FC0EAFF73
:10173000C80EEF6E1200D9CFE6FFE1CFD9FF020E3F
:10174000E126000EDE6E0D0EDD6EFD0EDB50E82490
:101750000D6EFE0EDB50040DF3500D24040DF3CF7F
:101760000BF0F4CF0CF0D9CFE9FFDACFEAFF0B5042
:10177000EE260C50ED22DECFE9FFDDCFEAFFEF9E33
:10178000FD0EDB500FE1FE0EEA6ADB34FE0BEA369B
:10179000E96E680EE926000EEA22DECFEEFFDDCF0D
:1017A000EDFF0ED0FE0EEA6ADB34FE0BEA36E96E80
:1017B0006E0EE926000EEA22DECFEEFFDDCFEDFF52
:1017C000DECFE9FFDDCFEAFFEF9CDECFE9FFDDCF23
:1017D000EAFF040EE926000EEA22EF8C020EE15C1D
:1017E00002E2E16AE552E16EE552E7CFD9FF12006D
:1017F0006598000178BF2BD07DAF09D0020E756FC0
:10180000945101E158DF0001926B916B1FD066C0CB
:10181000E9FF67C0EAFFEE52080EEF6E66C0E9FF0F
:1018200067C0EAFF020EE926000EEA22300EEE6ED5
:101830000D0EED6E66C0E9FF67C0EAFF8C0EEF6E1D
:101840006EC0E9FF6FC0EAFF840EEF6E31D00D016C
:1018500030AF0DD00001010E756F935101E12BDF08
:101860000001926B916B905101E1D4DE21D0000117
:10187000020E756F66C0E9FF67C0EAFFEE52080E00
:10188000EF6E66C0E9FF67C0EAFF020EE926000EB0
:10189000EA22300EEE6E0D0EED6E66C0E9FF67C0F7
:1018A000EAFF840EEF6E926B916B905101E1B2DE14
:1018B0001200D9CFE6FFE1CFD9FFE652080EDF6E66
:1018C0000001795D000E7A590BE279C0DFFF745197
:1018D00003E1010E746F04D0740502E1020E746F0F
:1018E000DF500B6E0C6A0B50795D796F0C507A5992
:1018F0007A6F6EC0E9FF6FC0EAFFEE52DFCFEFFFF5
:10190000380E826F0D0E836F78B119D0DF5016E05C
:1019100076C0F6FF77C0F7FF762B000E772308001E
:10192000F550E66E82C0E9FF83C0EAFF822B000E0D
:101930008323E552E750EF6EDF06E8D717D0DF507C
:1019400015E076C0E9FF77C0EAFF762B000E77231B
:10195000EF50E66E82C0E9FF83C0EAFF822B000EE3
:101960008323E552E750EF6EDF06E9D7E552E552F3
:10197000E7CFD9FF1200D9CFE6FFE1CFD9FF020EA2
:10198000E12664C0E9FF65C0EAFFEE52EFCFDFFF5A
:10199000DFCF0BF00B5000017E5D000E7F5902E29D
:1019A0007EC0DFFFDF500B6E0C6A0B507E5D7E6FDA
:1019B0000C507F597F6F010EDB6ADF50F36E010E12
:1019C000DBCFF4FFF350F45C16E2010EDB50EA6A61
:1019D000380FE96E0D0EEA22EF50E66E7BC0E9FF8C
:1019E0007CC0EAFF7B2B000E7C23E552E750EF6EB4
:1019F000010EDB2AE2D7000ED8807E55000E7F55FF
:101A000028E266C0E9FF67C0EAFFEE52080EEF6EFB
:101A100066C0E9FF67C0EAFF020EE926000EEA226F
:101A2000380EEE6E0D0EED6E64C0E9FF65C0EAFF84
:101A3000EF50400B07E166C0E9FF67C0EAFFC80E40
:101A4000EF6E06D066C0E9FF67C0EAFF880EEF6E52
:101A500028D066C0E9FF67C0EAFFEE52080EEF6EBD
:101A600066C0E9FF67C0EAFF020EE926000EEA221F
:101A7000300EEE6E0D0EED6E66C0E9FF67C0EAFF38
:101A8000840EEF6E8051811107E005D081C0FAFF0E
:101A900000018051F96EFADF00017D9F905101E154
:101AA000B9DD020EE15C02E2E16AE552E16EE55267
:101AB000E7CFD9FF1200D9CFE6FFE1CFD9FFE65239
:101AC0000001788F020EE66EE66AE66A270EE66E81
:101AD0000F0EE66E3CEC1AF00B6E050EE15E0B503D
:101AE000300EE66EE66AE66A000EE66E0D0EE66EF3
:101AF0003CEC1AF00B6E050EE15E0B50658CDF6A54
:101B0000030EDF5C10E2DF50EA6A890FE96E000E17
:101B1000EA22EF6ADF50EA6A8C0FE96E000EEA22D1
:101B2000EF6ADF2AEDD7020EE66EE66AE66A620E1B
:101B3000E66E000EE66E3CEC1AF00B6E050EE15EF2
:101B40000B50659C0001080E6E6F0D0E6F6F000E3E
:101B5000646F0D0E656F64C066F065C067F032CDCE
:101B600061F0615103E1100E606F13D0010EE66E5B
:101B7000E66A610EE66E000EE66E010EE66EE66A3D
:101B8000ADEC16F00B6E060EE15E0B500001200E60
:101B9000606FE552E552E7CFD9FF1200800E0D01CC
:101BA000305D5BE10001C00E786F0D013351030A17
:101BB00034E0010A0EE0030A03E00001786B4DD027
:101BC0000001D20E766F320E776F120E796F7A6B3C
:101BD00044D03251F66EF76AD890F636F736930E47
:101BE000F626330EF7220900F5CF76F00A00F5CF7E
:101BF00077F0020E0001F76A7625F66E7751F7222C
:101C00000800F5CF79F0030EF76A7625F66E775166
:101C1000F7220800F5CF7AF020D0030E325D1AE2E9
:101C20003251F66EF76AD890F636F736950EF626EC
:101C3000330EF7220900F5CF76F00A00F5CF77F0E2
:101C400076C0F6FF77C0F7FF0800F5500001796F06
:101C50007A6B02D00001786B00D01200D9CFE6FF7A
:101C6000E1CFD9FF020EE1260D01386B396B3051FF
:101C70001F0B020A12E0030A0DE0010A01E042D044
:101C80000001788F0D0138810001840502E10D010A
:101C9000388338D00001788F35D00001788F0D015E
:101CA00034BF10D034510F0BE96EEA6AD890E93690
:101CB000EA36680EE926000EEA22EECFDEFFEDCF0F
:101CC000DDFF0FD034510F0BE96EEA6AD890E93688
:101CD000EA366E0EE926000EEA22EECFDEFFEDCFE9
:101CE000DDFFDECFE9FFDDCFEAFFEF50800B09E03B
:101CF000DECFE9FFDDCFEAFFEF50040B02E0010E7B
:101D0000386F00D0000178AF07D0380E766F0D0E17
:101D1000776F7881020E796F020EE15C02E2E16A70
:101D2000E552E16EE552E7CFD9FF12000F0126A17F
:101D300015D064C0E9FF65C0EAFFEF5080080DE1EF
:101D40006EC0E9FF6FC0EAFFEF50840806E164C08F
:101D5000E9FF65C0EAFF8C0EEF6E2691629A1200D1
:101D60000F013685629865820001010E856F000EB5
:101D7000E66EE66AE66EE66A750EE66EE66AADEC5B
:101D800016F00B6E060EE15E0B5012000001856B23
:101D9000000EE66EE66AE66EE66A740EE66EE66AC7
:101DA000ADEC16F00B6E060EE15E0B5065920F0166
:101DB000369562A402D06294FCD71200D9CFE6FF18
:101DC000E1CFD9FFE65200012D0E8F6FFD0E861573
:101DD00053E17E0E8615E8407F0B040DF3CF64F0CF
:101DE000F4CF65F0000E64270D0E652364C066F025
:101DF00065C067F0667564C0E9FF65C0EAFFEF5033
:101E00003C0BE842E8420D0835E1DF6A080EDF5C72
:101E100023E264C0E9FF65C0EAFF020EE926000E76
:101E2000EA22EE50EFCFEAFFE96EEF50E66EDF50A8
:101E3000EA6A300FE96E0D0EEA22E552E750EF6EC6
:101E400064C0E9FF65C0EAFF020EE926000EEA223F
:101E5000EE2AEF22DF2ADAD764C0E9FF65C0EAFF85
:101E6000020EE926000EEA22300EEE6E0D0EED6E29
:101E70000DD801D03AD805D0FD0E8615040801E131
:101E800059D8E552E552E7CFD9FF12000001746B33
:101E9000906B936B946B886B756B6EC0E9FF6FC032
:101EA000EAFFEF9E6E756EC0E9FF6FC0EAFFEF9E1E
:101EB0006E7566C0E9FF67C0EAFFEF9E786B796BCD
:101EC0007A6B7D6B7E6B7F6B92D8000EE66EE66A56
:101ED000E66EE66A030EE66EE66AADEC16F00B6E91
:101EE000060EE15E0B50F8EF0BF0020E0001755D7F
:101EF00002E141DD1ED0756B88511AE166C0E9FF31
:101F000067C0EAFFEE52080EEF6E66C0E9FF67C0D9
:101F1000EAFF020EE926000EEA22300EEE6E0D0EEA
:101F2000ED6E66C0E9FF67C0EAFF8C0EEF6E01D070
:101F3000886B1200D9CFE6FFE1CFD9FFE6526EC021
:101F4000E9FF6FC0EAFFEF50400B01E0010EDF6ECA
:101F500000016E75080E605D0CE132CD38FF0F0197
:101F6000385104E00001100E606F03D00001040E30
:101F7000606F750528E16EC0E9FF6FC0EAFF020ED1
:101F8000E926000EEA22380EEE6E0D0EED6E91DCA3
:101F9000020E0001745D07E16EC0E9FF6FC0EAFF49
:101FA000840EEF6E0FD0DF5007E16EC0E9FF6FC007
:101FB000EAFFC80EEF6E06D06EC0E9FF6FC0EAFF01
:101FC000880EEF6E0FD07DAF0CD08051811107E0ED
:101FD00005D081C0FAFF00018051F96EFADF0001DF
:101FE0007D9F756BE552E552E7CFD9FF12000D01D9
:101FF0003051600BE842E842E842E842E84200091A
:1020000001E058D031510C0A54E00B0A43E00C0AAD
:1020100035E0010A26E00B0A22E0020A20E0030A6A
:102020001CE0080A10E0010A0CE00F0A08E0030AAD
:1020300001E03FD00001788F080E606F3BD0AEDD2D
:1020400039D039DD37D00001610E766F000E776F21
:102050007881010E796F788F2DD000DE2BD02BD8B0
:1020600029D034510001766F776B620E7627000E0F
:1020700077237881010E796F788F1CD00001788FDB
:102080000D013451EA6A620FE96E000EEA2232CD88
:10209000EFFF10D0000EE66EE66AE66EE66A020E0C
:1020A000E66EE66AADEC16F00B6E060EE15E0B50C6
:1020B00001D000D01200D9CFE6FFE1CFD9FF050E45
:1020C000E1260D01320510E130511F0B00090CE132
:1020D0000001788F030E0D01315D04E10001010E56
:1020E000846F02D00001846B0D01325101E020D1D8
:1020F00030511F0B020801E01BD134510F0B0009B6
:1021000001E116D134510F0B020801E211D1200E6A
:102110000001605D01E00CD1788F0D0134BF1AD051
:1021200034510F0BE96EEA6AD890E936EA36680E48
:10213000E926000EEA22EECFDEFFEDCFDDFF3451BF
:102140000F0BEA6A8C0FE96E000EEA22020EEFCF47
:10215000DBFF19D034510F0BE96EEA6AD890E936EB
:10216000EA366E0EE926000EEA22EECFDEFFEDCF54
:10217000DDFF34510F0BEA6A890FE96E000EEA2287
:10218000020EEFCFDBFFD950020FE96EDACFEAFF84
:10219000EF50010B03E1000EDF9401D0DF8434BF68
:1021A00010D034510F0BE96EEA6AD890E936EA365E
:1021B000680EE926000EEA22DECFEEFFDDCFEDFF4E
:1021C0000FD034510F0BE96EEA6AD890E936EA363F
:1021D0006E0EE926000EEA22DECFEEFFDDCFEDFF28
:1021E000030E315D23E1DECFE9FFDDCFEAFFEF50E3
:1021F000800B13E034BF09D034510F0BEA6A8C0F07
:10220000E96E000EEA22EF8208D034510F0BEA6A21
:10221000890FE96E000EEA22EF82840E0B6EDECF8C
:10222000E9FFDDCFEAFF0B50EF1282D0DF74DECF83
:10223000E9FFDDCFEAFFEF50800B1BE0DECFE9FFC7
:10224000DDCFEAFFEF9EDECFE9FFDDCFEAFFEF8CC7
:10225000020EE66EE66ADECFE6FFDDCFE6FF050E94
:10226000E66EE66AADEC16F00B6E060EE15E0B5004
:1022700005D0DECFE9FFDDCFEAFFEF8CDF74D95068
:10228000020FE96EDACFEAFFEF50020B07E1DECF73
:10229000E9FFDDCFEAFFEF50800B2DE00D0134BFE9
:1022A00009D034510F0BEA6A8C0FE96E000EEA2256
:1022B000EF9208D034510F0BEA6A890FE96E000ED5
:1022C000EA22EF923B0E0B6EDECFE9FFDDCFEAFF95
:1022D0000B50EF16020EE66EE66ADECFE6FFDDCFAC
:1022E000E6FF050EE66EE66AADEC16F00B6E060E26
:1022F000E15E0B5008D03B0E0B6EDECFE9FFDDCF69
:10230000EAFF0B50EF160D0134510F0B0C6A260F2C
:102310000B6E0F0E0C22030E0BC0DBFF040E0CC065
:10232000DBFF030EDBCFE9FF040EDBCFEAFFEF900C
:10233000050EE15C02E2E16AE552E16EE552E7CFAB
:04234000D9FF1200AF
:0C234400DACFE4FFE2CFDAFFE652E55208
:10235000E5CFDAFF1100D8CFE4FFE0CFE4FFE46E71
:10236000DACFE4FFE2CFDAFFE652E552E5CFDAFF5B
:10237000E550E5CFE0FFE5CFD8FF100005D8ACEC85
:1023800008F0D9D8FCD71200D9CFE6FFE1CFD9FFAA
:10239000020EE1260F0EC112580EDE6E020EDD6E29
:1023A0009B8CDFCF0BF0DF06010EDBCF0CF001E2E0
:1023B000DB060B500C1001E0F4D70F017F0E486FC5
:1023C000BF0E496F0CD81CEC08F0020EE15C02E273
:1023D000E16AE552E16EE552E7CFD9FF1200D9CFAD
:1023E000E6FFE1CFD9FFE65236D8AD8CAC8C948CA9
:1023F0008B9C0F014181938E939C0E01060EC96F39
:102400000A0EF76F240EA86E900E9C6E710EAB6EC6
:10241000020E7D6E380E7C6EDF6ADF500B6E0C6A2A
:10242000400E0B5C000E0C5809E2DF50EA6A000F08
:10243000E96E010EEA22EF6ADF2AEFD70101806B15
:10244000816B836B846BFC0E8D169616E552E552FC
:10245000E7CFD9FF1200D9CFE6FFE1CFD9FFE6528F
:10246000948E949C240EAD6E900EAC6E710EB06E78
:10247000020E7F6E080E7E6EAF50DF6EE552E552A3
:10248000E7CFD9FF1200D9CFE6FFE1CFD9FFFE0E8B
:10249000DBCFE6FFDB407F0B116EFE0EDB40E8403A
:1024A0003F0B106EFE0EDB40E840E8401F0B0F6E46
:1024B000FE0EDB380F0B0E6EFE0EDB50E00BE83825
:1024C000E8400D6E060E0C6EFE0EDB500CC0E7FFF2
:1024D000E75204E0E8427F0BE706FCE10B6EFE0EDC
:1024E000DB44010B0B180D180E180F1810181118DB
:1024F000E552E718010BE8B0AD80E8A0AD90FE0E04
:10250000DB50AE6EE552E7CFD9FF1200D9CFE6FF20
:10251000E1CFD9FFE652ACA205D0AC98AF50DF6E48
:10252000AC8802D0AF50DF6EDF5000D0E552E552EC
:10253000E7CFD9FF1200D9CFE6FFE1CFD9FF040ED4
:10254000E126200E0001E76E6019E8AE02D0E73404
:1025500002D0E750605D03E36550020B01E082D3D7
:102560000101E0510B6E0C6AD8900C5004E6FA0E93
:102570000B5C000E0C5801E2E02BE0510B6E0C6A74
:10258000FA0E0B1801E10C5001E1DE6BE1510B6E0C
:102590000C6AD8900C5004E6FA0E0B5C000E0C5836
:1025A00001E2E12BE1510B6E0C6AFA0E0B1801E10E
:1025B0000C5001E1DF6BDD0502E1FE0EDF6FACA226
:1025C00002D0AC98AC88ACA403D0020EAFCFDBFF36
:1025D0009CA202D09C989C889CA403D0030EAACFF6
:1025E000DBFFA4AA73D01DEC1AF00101D86F800E96
:1025F000D85D03E10101010EE66F400E0101D85DD7
:1026000002E10101E66B020E0101E65D05E1010157
:10261000D85102E00101E66B030E0101E65D02E123
:10262000D8C1D9F1040EE65D06E1200E0101D80300
:10263000F350D925D96F050E0101E65D0EE10101C8
:10264000D8510B6E0C6A060ED8900B360C36E80487
:10265000FBE10BC0E7F10CC0E8F1060E0101E65DFD
:1026600034E10101D8510101E711E76F0101D951AE
:102670000101E95D07E3D9C1E9F1E7C1D0F1E8C1A2
:10268000D1F123D00101D9510101EA5D07E3D9C19C
:10269000EAF1E7C1D2F1E8C1D3F117D00101D95174
:1026A0000101EB5D07E3D9C1EBF1E7C1D4F1E8C16A
:1026B000D5F10BD00101D9510101EC5D06E3D9C17F
:1026C000ECF1E7C1D6F1E8C1D7F1E62BDC5101E02E
:1026D00059D1400EE66E400EE66E010EE66EC6EC77
:1026E00017F0E552E552E5520101816F8151000872
:1026F00001E348D10101E06BDF6B030EE76EDE19E9
:10270000E8AE02D0E73402D0E750DE5D01E335D118
:1027100081C1DFFFDFCF0BF0030EE76E0B18E8AED1
:1027200002D00B3403D0E750D8800B5402E2030EE2
:10273000DF6E010EDB6ADBCF0BF0DF50E76E0B18AC
:10274000E8AE02D0E73402D0E7500B5C1CE2010E89
:10275000DBCFE9FFEA6AE9BEEA68400EE926010E2E
:10276000EA22EF50E66EDEC1E9FFEA6AE9BEEA68F6
:10277000850EE926010EEA22E552E750EF6EDE2BC8
:10278000010EDB2AD8D7020EE76EDE19E8AE02D0C2
:10279000DE3503D0E750D880DE5531E201018505F2
:1027A0002EE1020E865D2BE1FC0E875D28E1010122
:1027B000010EDD6F01018051EA6A000FE96E010E22
:1027C000EA22010EEF6E802B8051EA6A000FE96E5B
:1027D000010EEA22030EEF6E802B8051EA6A000F91
:1027E000E96E010EEA22010EEF6E802B8051EA6A3B
:1027F000000FE96E010EEA22FA0EEF6E802B020E38
:102800000101E76EDE19E8AE02D0DE3503D0E750F5
:10281000D880DE5501E3B1D00101855101E0ADD092
:10282000020E865D01E0A9D0FD0E875D01E0A5D016
:102830000101010EDD6FE36901018051EA6A000FB9
:10284000E96E010EEA22EF6A8051EA6A000FE96E32
:10285000010EEA22EF500101E35DE36F0101802BDD
:102860008051EA6A000FE96E010EEA22060EEF6E51
:102870008051EA6A000FE96E010EEA22EF50010171
:10288000E35DE36F0101802BFF0ED880D055000E71
:10289000D15502E2D069D16B8051EA6A000FE96E2E
:1028A000010EEA22D0C1EFFF8051EA6A000FE96E03
:1028B000010EEA22EF500101E35DE36F0101802B7D
:1028C000FF0ED880D255000ED35502E2D269D36BE9
:1028D0008051EA6A000FE96E010EEA22D2C1EFFFD1
:1028E0008051EA6A000FE96E010EEA22EF50010101
:1028F000E35DE36F0101802BFF0ED880D455000EFD
:10290000D55502E2D469D56B8051EA6A000FE96EB1
:10291000010EEA22D4C1EFFF8051EA6A000FE96E8E
:10292000010EEA22EF500101E35DE36F0101802B0C
:10293000FF0ED880D655000ED75502E2D669D76B68
:102940008051EA6A000FE96E010EEA22D6C1EFFF5C
:102950008051EA6A000FE96E010EEA22EF50010190
:10296000E35DE36F0101802B8051EA6A000FE96E9D
:10297000010EEA22E3C1EFFF802B0101010EDC6FA3
:102980000101826B0101DC5115E0AD50020B12E038
:1029900001018251EA6A400FE96E010EEA22EF500E
:1029A000E66E71DDE5520101822B8151825D02E10B
:1029B0000101DC6B9E50200B01E13ED13F0E010175
:1029C000805D01E339D1A2DDE66E01018051EA6A42
:1029D000000FE96E010EEA22E552E750EF6E0101A9
:1029E000E16BDE6B01018051EA6A000FE96E010EB6
:1029F000EA22EF50E66EDFC1E9FFEA6AE9BEEA6863
:102A0000940EE926010EEA22E552E750EF6E010E20
:102A10000101E76EDF19E8AE02D0DF3503D0E750E1
:102A2000D880DF550EE2E251DF5D0BE201018051FB
:102A3000EA6A000FE96E010EEA22EF500101E35D40
:102A4000E36FDF0526E1F00E0101945D22E1805184
:102A5000EA6A000FE96E010EEA22EFCFE2F101010E
:102A60000F0EE36F080EE225E66E01018051EA6A5F
:102A7000000FE96E010EEA22E552E750EF6E805139
:102A8000EA6A000FE96E010EEA22EF500101E35DF0
:102A9000E36F0101E251DF5D01E0B9D0F00E010109
:102AA000945D01E0B4D08051EA6A000FE96E010E36
:102AB000EA22D0C1EFFF8051EA6A000FE96E010EF1
:102AC000EA22EF500101E35DE36F0101802BD1C1E8
:102AD0000BF00C6A8051EA6A000FE96E010EEA22DF
:102AE0000BC0EFFF8051EA6A000FE96E010EEA2287
:102AF000EF500101E35DE36F0101802B8051EA6A31
:102B0000000FE96E010EEA22D2C1EFFF8051EA6A9E
:102B1000000FE96E010EEA22EF500101E35DE36F61
:102B20000101802BD3C10BF00C6A8051EA6A000FBF
:102B3000E96E010EEA220BC0EFFF8051EA6A000F36
:102B4000E96E010EEA22EF500101E35DE36F01013E
:102B5000802B8051EA6A000FE96E010EEA22D4C18F
:102B6000EFFF8051EA6A000FE96E010EEA22EF5092
:102B70000101E35DE36F0101802BD5C10BF00C6A0D
:102B80008051EA6A000FE96E010EEA220BC0EFFFE6
:102B90008051EA6A000FE96E010EEA22EF5001014E
:102BA000E35DE36F0101802B8051EA6A000FE96E5B
:102BB000010EEA22D6C1EFFF8051EA6A000FE96EEA
:102BC000010EEA22EF500101E35DE36F0101802B6A
:102BD000D7C10BF00C6A8051EA6A000FE96E010E52
:102BE000EA220BC0EFFF8051EA6A000FE96E010E86
:102BF000EA22EF500101E35DE36F0101802B805178
:102C0000EA6A000FE96E010EEA22E3C1EFFF3B0E14
:102C10000101E76EDF19E8AE02D0E73402D0E750D9
:102C2000DF5D01E2DF2B0101802B8051EA6A000F9A
:102C3000E96E010EEA22EF6A0E01925111E10101E3
:102C4000805100080DE280C1E6FF000EE66E010E25
:102C5000E66E27EC18F0E552E552E5520101806B73
:102C6000C3EC18F0040EE15C02E2E16AE552E16EA9
:102C7000E552E7CFD9FF12000101ED51EE1104E159
:102C8000100EED6F270EEE6FED07000EEE5B65A2E6
:102C90000AD0ED51EE1106E18D708DA002D08D822B
:102CA00001D08D922ED00001605103E18D908D9264
:102CB00028D0600503E18D808D8223D0020E605DF7
:102CC00003E18D808D921DD0040E605D03E18D9037
:102CD0008D8217D0100E605D07E10101ED51EE11FC
:102CE00002E18D708D920DD0200E605D0AE1010130
:102CF000ED51EE1106E18D708DA002D08D9201D0C4
:102D00008D8212001200120012001200FCEF16F069
:102D100012004DEF17F0000184051EE1000185054A
:102D20001BE1F1DF65920001856B0101100EDA6F86
:102D30000E0EDB6FDA07000EDB5BDA51DB11FAE116
:102D40006584080EDA6F070EDB6FDA07000EDB5BB7
:102D5000DA51DB11FAE165941200D9CFE6FFE1CF39
:102D6000D9FFFD0EDBCF06F0FE0EDBCF07F0050E20
:102D7000061801E1075039E0E868061802E17F0E05
:102D8000071831E0030E061801E107502AE0020E91
:102D9000061801E1075023E0010E061801E1075073
:102DA0001CE0740E061801E1075015E0750E0618B8
:102DB00001E107500EE0730E061801E1075007E02D
:102DC000720E061801E1075001E010D00FD09CDF11
:102DD0000DD098DF0BD097DF09D09BDF07D098DFAD
:102DE00005D094DF03D091DF01D000D0010E00D0D8
:082DF000E552E7CFD9FF120004
:082DF8000D0130511F0B010811
:102E000001E04AD03051600BE842E842E842E84233
:102E1000E842010801E040D0345103E0340501E00C
:102E20003BD03151220A33E0030A26E0010A17E0C1
:102E3000210A0EE0010A01E02FD00001A20E766FF8
:102E40000E0E776F080E796F7A6B7881788F24D0A9
:102E50000001A20E766F0E0E776F788F1DD036CDE3
:102E60007EF037CD7FF00001800E7B6F0E0E7C6F01
:102E7000806B816B7D8F10D00001800E766F0E0EFF
:102E8000776F070E796F7A6BC10E786F05D032CDF0
:102E90009DFE0001788F00D012000E01806B4B0E5A
:102EA000816F826B836B846B856B080E866F916B71
:102EB0001A0EE66E010EE66E88EC09F0E552E55258
:102EC0001E0EE66E020EE66E88EC09F0E552E55243
:102ED000400EE66E400EE66E0E0EE66EE66A020EDE
:102EE000E66EBFEC09F00B6E050EE15E0B50F3CF02
:102EF00099FEF4CF9AFE0E019B6B9C6B926B1200B5
:102F0000D9CFE6FFE1CFD9FFFD0EDBCF06F0FE0EF5
:102F1000DBCF07F0050E061801E1075002E0000EB6
:102F200031D0FB0EDBCF0BF0FC0EDBCF0CF00E0133
:102F300099510B1802E19A510C1813E1400EE66EFC
:102F4000400EE66E0E0EE66EE66A020EE66EBFEC10
:102F500009F00B6E050EE15E0B50F3CF99FEF4CF36
:102F60009AFEFB0EDBCF0BF0FC0EDBCF0CF00E015C
:102F70009B510B1802E19C510C1802E1926B976B6C
:102F8000010E00D0E552E7CFD9FF1200D9CFE6FFFE
:102F9000E1CFD9FF0E01916B99519A1102E1000E18
:102FA00008D099CEE9FF9ACEEAFFEF50800B01E0FE
:102FB000010E000945E1FC0EDBCF0BF099CEE9FFD5
:102FC0009ACEEAFFEE52EF50D8800B5408E299CE29
:102FD000E9FF9ACEEAFFEE52FC0EEFCFDBFF916BDA
:102FE000FC0EDB50915D19E29151EA6A400FE96EE7
:102FF0000E0EEA22EF50E66E9151E76EFD0EDBCF2A
:10300000E9FFFE0EDBCFEAFFE750E926000EEA22D9
:10301000E552E750EF6E912BE3D7400EE66E400E7F
:10302000E66E0E0EE66EE66A020EE66EBFEC09F084
:103030000B6E050EE15E0B50F3CF99FEF4CF9AFEB6
:103040000E01915100D0E552E7CFD9FF1200D9CF40
:10305000E6FFE1CFD9FF0E0192510CE1FD0EDBCF6F
:1030600093FEFE0EDBCF94FEFC0EDBCF97FE010E2F
:10307000986F926FE552E7CFD9FF1200D9CFE6FFE4
:10308000E1CFD9FF030EE1260E01925101E02ED0CF
:10309000DF6AFD0EDBCF06F0FE0EDBCF07F0DE525F
:1030A00006C0DEFF07C0DDFFDD52DF2ADF500B6EFA
:1030B0000C6AFF0E0B1801E10C5001E10BD0010E60
:1030C000DBCFE9FFDB2A020EDBCFEAFF01E3DB2ADD
:1030D000EF50EBE1FD0EDBCF93FEFE0EDBCF94FE57
:1030E000DFCF97FE0E01010E986F926F030EE15C29
:1030F00002E2E16AE552E16EE552E7CFD9FF120044
:10310000D9CFE6FFE1CFD9FF030EE1260E019251A0
:1031100001E02FD0DF6AFD0EDBCF06F0FE0EDBCF25
:1031200007F0DE5206C0DEFF07C0DDFFDD52DF2AFA
:10313000DF500B6E0C6AFF0E0B1801E10C5001E121
:103140000CD0010EDBCFF6FFDB2A020EDBCFF7FF40
:1031500001E3DB2A0800F550EAE1FD0EDBCF93FE28
:10316000FE0EDBCF94FEDFCF97FE0E01986B010EB3
:10317000926F030EE15C02E2E16AE552E16EE55214
:10318000E7CFD9FF1200D9CFE6FFE1CFD9FF020E7A
:10319000E1260E019B519C1102E1000E08D09BCE4E
:1031A000E9FF9CCEEAFFEF50800B01E0010E000921
:1031B00001E085D0030E925D01E1926B925101E135
:1031C0007ED0020E925D16E1E66A000EE66EE66AB9
:1031D000010EE66E020EE66EBFEC09F00B6E050EF8
:1031E000E15E0B50F3CF9BFEF4CF9CFE0E01030E6D
:1031F000926F65D0920563E1400E0B6E0C6A975199
:103200000B5C000E0C5803E2400EDF6E02D097CE2E
:10321000DFFFDF50975D976F000E956F0E0E966F74
:10322000010EDFCFDBFF985117E1010EDB5013E0F9
:1032300093CEF6FF94CEF7FF0800F55095CEE9FF48
:1032400096CEEAFFEF6E952B000E9623932B9423D8
:10325000010EDB06EAD715D0010EDB5012E093CE4B
:10326000E9FF94CEEAFFEF5095CEE9FF96CEEAFF54
:10327000EF6E952B000E9623932B9423010EDB0605
:10328000EBD7975108E1400EDF5C03E1020E926F2D
:1032900002D0030E926FDFCFE6FF000EE66E0E0E39
:1032A000E66E010EE66E020EE66EBFEC09F00B6EE6
:1032B000050EE15E0B50F3CF9BFEF4CF9CFE020E99
:1032C000E15C02E2E16AE552E16EE552E7CFD9FF47
:0232D0001200EA
:0E32D2001201000202000008D8040A000001E8
:1032E0000102000109024300020100C0320904008A
:1032F000000102020100052400100104240202055D
:10330000240600010524010001070581030A0001CC
:1033100009040100020A0000000705020240000043
:10332000070582024000000403090434034D0069CC
:1033300000630072006F0063006800690070002085
:103340000054006500630068006E006F006C006F41
:103350000067007900200049006E0063002E0034F1
:10336000034300440043002000520053002D00326C
:103370000033003200200045006D0075006C0061D4
:1033800000740069006F006E002000440065006D4D
:0B339000006F00E43227332B335F3363
:04339C002A0EF66E91
:1033A000100EF76E000EF86E01010900F550F46F73
:1033B0000900F550F56F03E1F46701D03DD0090035
:1033C000F550EF6F0900F550F06F0900F550F16FFF
:1033D00009000900F550E96E0900F550EA6E090090
:1033E00009000900F550F26F0900F550F36F09006C
:1033F0000900F6CFF6F1F7CFF7F1F8CFF8F1EFC10A
:10340000F6FFF0C1F7FFF1C1F8FF0101F25302E14D
:10341000F35307E00900F550EE6EF207F8E2F30708
:10342000F9D7F6C1F6FFF7C1F7FFF8C1F8FF0101C0
:0A343000F407000EF55BBFD7120091
:06343A00D9CFE6FFDACF56
:10344000E6FFE1CFD9FFE2CFDAFFE652F20E0E013E
:10345000AA179CAC03D0AA919CB0AA819CB4AA855F
:103460009CB2AA87AA50DF6EDF50E552E552E5CF45
:08347000DAFFE7CFD9FF1200DB
:08347800FE0EE3CFE9FFFF0E99
:10348000E3CFEAFFE9CFF3FFEACFF4FFFB0EE3500F
:1034900003E1FC0EE35009E0FB0EE30602E2FC0E42
:0C34A000E306FD0EE350EE6EF1D71200C3
:0434AC00B00EF36EFD
:1034B00000EE00F00E0E01D81200EA6002D0EE6AB3
:0C34C000FCD7F350E9601200EE6AFCD764
:0434CC001CEE00F002
:1034D0002CEE00F0F86A0A9CCEEC19F074EC1AF0AD
:0834E000BEEC11F0FBD7120055
:0234E8001200D0
:0634EA00000000000000DC
:0D34F000FF000000000000FFFFFFFF0000D4
:020000040001F9
:01FFF800BC4C
:01FFF900F710
:01FFFA003ACC
:01FFFB00FF06
:01FFFC0063A1
:01FFFD00FA09
:01FFFE008181
:01FFFF00F908
:00000001FF
